:030000000219FDE5
:03000B000200AA46
:03002B0002015C73
:03005B000202F9A5
:030073000202E6A0
:1000800002030406080C10182030406080040608A3
:100090000C10182030406080A0C00003070F1F0D17
:1000A0000D04050D050305030302C2AFC0D0C0E077
:1000B000206214E5256009E473E525F4F58AD2622F
:1000C000D0E0D0D0D2AF3285268AC262E526F46075
:1000D0002F30682520720DD0E0D0D0C293C295C2D7
:1000E00097D2AF32C293C295C297206F0C20660997
:1000F000740AD5E0FDE57B4290D0E0D0D0D2AF329B
:10010000758A00C28DD26201F901B9306805206696
:1001100002D29301B9306805206602D29501B93048
:100120006805206602D29701B9C29230680A20663B
:10013000077408D5E0FDD29301B9C29430680A2053
:1001400066077408D5E0FDD29501B9C29630680AF9
:100150002066077408D5E0FDD29701B9C2AFC2ADE1
:1001600053E6EFC0D0C0E0D2D3D2AFC2CEE52A6012
:1001700007207449152A21BD7800790020742EE5E6
:1001800080307E01F430E30278FF53DACF207E0323
:1001900043DA20307E0343DA10C2D8C271E58030E2
:1001A0007E01F430E30279FFC3E89970CB3061033C
:1001B000752A18207403752A18885CD27020740D73
:1001C000E52B6004152B21CD43DA01C2D820700243
:1001D000413CA85C206102C2702074367982B70469
:1001E00031C3E894F0400374F0F8E8C4540F28F8E1
:1001F0007984B703024112C313C313872120080275
:10020000C313200A06C3C898F8411228F850037493
:10021000FFF88822E52D54066022206B1FE536C3C7
:1002200033C333F8E564C313C313F9C39522400203
:100230008922E82522F52250037522FF7882B60430
:1002400059852224A824C3E52495614002A861C3EE
:10025000E895634002A8638825E5667002418DC376
:10026000E8AA669A5003E8FAE4F9EAC333FBE568C2
:10027000F45B29400D2567F8E56760021567400BC0
:10028000418D0AC3E5679A5002056778FF8826C248
:100290006FC3E52694F84002D26FC3E52594404031
:1002A00002D26420CF0AD0E0D0D043E610D2AD32E3
:1002B000C2CF053A7801E52A6005307402152AC3D9
:1002C000E55C94014005755F0041DC75600075696F
:1002D00000E55F2401F55F5003755FFFD0E0D0D0EB
:1002E00043E610D2AD32C2AF53E67F7592FA7593F2
:1002F000FFC260759104D2AF32C2AF53E6EFC2AD18
:10030000C0D0C0E0C0F0D2D3D2AFA8FBA9FCC2D805
:10031000307102616053DACF207E0343DA10307E01
:100320000343DA20D271E580307E01F420E30261DC
:100330003788278928A18D53DACF207E0343DA201E
:10034000307E0343DA10C2D8C271307402A17978CA
:1003500000E580307E01F430E302A179885CA16180
:1003600053DACF207E0343DA20307E0343DA10C213
:1003700071206102813953DACF207E0343DA1030D5
:100380007E0343DA20C2D8D27188578958C3E895D2
:1003900055F8E99556F97B007E087A00C3E8948CFD
:1003A000E994005005755B00812B882178A2E6A8AE
:1003B000216055C3E894C8E994005008E4D2E4FBF6
:1003C0007A0A8106C3E89468E994015008E4D2E30C
:1003D000FB7A0F8106C3E894D0E994025008E4D276
:1003E000E2FB7A1E8106C3E894A0E994055008E474
:1003F000D2E1FB7A3C8106C3E89498E9940850085E
:10040000E4D2E0FB7A787E00C3E89559FCE9955A7E
:10041000FD30E70AECF42401FCEDF43400FD755BDB
:1004200000C3EC9AED9E5003755B018859895A858B
:1004300057558558567802A161C3E89527F8E99584
:1004400028F9307C02A145307B02A145307A02A117
:100450003E207502815CE9FDE8FC817BE9C313F96C
:10046000E813F8307902A13EE9C313F9E813F83034
:0F0470007802A13EE9C313FDE813FC20612CC301
:10047F00EC941CED940240028192ED701EC3EC943B
:10048F00C850180529E52970021529C3E529940AD2
:10049F005002A179755C00D270A179E5296002152F
:1004AF00297888E6F97400207F087896B9030278D6
:1004BF009EE624FAFEE43400FFC3EC9EFCED9FFDA4
:1004CF009208B90310A2085007207609D27681E46A
:1004DF00307602C276A2085016B9030DECF424014F
:1004EF00FCEDF43400FD0204FE78007900A145B95B
:1004FF000315EC33FCED33FDC3EC940AFCED9400D3
:10050F00FD50047C007D00C3EC94FFED9400400689
:10051F0078FF7900A145EC8572F0A4C5F0A2F733FE
:10052F00F87900400302056178FF7900020561E95F
:10053F00C313F9E813F8307C0EE9600278FFC3E8C3
:10054F001338F8E43400F9C3E894FFE9940040024B
:10055F0078FF885CD270206102A179741FF4552F47
:10056F004BF52FC274EB7002D274752A18307403D6
:10057F00752A0A306102A18D20740353DAFE2074AC
:10058F0003752B06D0F0D0E0D0D0D2AD43E61032B9
:10059F0079010205BD79030205BD790A0205BD790E
:1005AF001E0205BD79640205BD79C80205BD781725
:1005BF00E4D5E0FDD8FAD9F6227A147B780205E467
:1005CF007A107B8C0205E47A0D7BB40205E47A0B7A
:1005DF007BC80205E47902E4C294D5E0FDD295D53B
:1005EF00E0FDC295D5E0FDD294D5E0FDE920E00213
:1005FF00D29330E002D297E573D5E0FDE920E00217
:10060F00C29330E002C2977496D5E0FDD9C9EAF8DB
:10061F00D5E0FDD8FBDBBEC29422C37C007D007504
:10062F00F00005F0EA33FAEB33FB50F6EB13FBEA7D
:10063F0013FAC3E9FFE8FEE89AF8E99BF95004EFD3
:10064F00F9EEF8B3EC33FCED33FDD5F0DFEDF9EC5B
:10065F00F822E889F08A20D2D4F8A9F07B0030F78D
:10066F000B7BFFF42401F8E9F43400F9E88520F05E
:10067F00A4ADF0F8E98520F0A4AFF0FEED2EF974EB
:10068F00003FFA7C04C3EA13FAE913F9E813F8DC24
:10069F00F48BF030F70AE8F42401F8E9F43400F9A8
:1006AF00E889F0C2D4F8A9F0227882B604030207D1
:1006BF0013C3E55C940140030206DD852224E4F5B3
:1006CF0044F545F546F547F548C26E0207137882A3
:1006DF00E6FCD26EE522F523783879C7AA40AB4104
:1006EF00C3EB13FBEA13FAEC146013C3EB13FBEA2F
:1006FF0013FAEC14146007C3EB13FBEA13FAD129B6
:10070F008844894522C3E5449523F8E5459400F9CB
:10071F00500CC3E89480E994FF4016020744C3E8E5
:10072F00947FE994005003020744787F7900020711
:10073F0044788079FF8849894A22E5492546F8E5BA
:10074F004A3547F9854A20E4300701F43548FA3035
:10075F00E709C3EA94F04015020782C3EA940F50E9
:10076F000302078278FF79FF7A0F020782780079F8
:10077F00007AF0C3E5249561500AC37401952450A3
:10078F000B0207A0E54A20E70E0207A0E54A30E773
:10079F0006884689478A482278A5E6FAC3E5493391
:1007AF00F8E54A33F9D161E930E70BC3E89480E902
:1007BF0094FF4013E1DAC3E8947FE994005002E11B
:1007CF00DA787F7900E1DA788079FFE820E715C3DE
:1007DF00E52398F84009C3E8940140030208017823
:1007EF0001020801E8F424012523F840030208015F
:1007FF0078FF884B2278A6E6FAA847A94812066127
:10080F00E930E70CC3E89401E994FF40160208367B
:10081F00C3E894FFE99400500302083678FF79008B
:10082F00020836780179FFE920E715C3E54B98F800
:10083F004009C3E89401400302085D780102085D96
:10084F00E8F42401254BF8400302085D78FF882463
:10085F002278FFC26420693D206A12D264C3E54149
:0F086F00940A4009C3E52594405002C26479A160
:10087E00E76023E541601F74FF8541F0848539F000
:10088E00306A0375F005A4F8C5F0600278FFC3E87E
:10089E0095645002A864886322C3E5409440E54104
:1008AE009401E56350031401B8046002F56322025B
:1008BE0008C02275E890227883E6FFE5E820ECF781
:1008CE00A8BDA9BE0570C3E57094084052757000AE
:1008DE00E9FA79A0E76044EA7007E571601B020847
:1008EE00FBC3E895716010E5715006600C140209A7
:1008FE00070460F9020907E571F571C394A8401B5E
:10090E007561C0C394054013756180C39405400B97
:10091E00756140C39405400375610075BB0122E506
:10092E00612410500274FFF5617982B704022154DC
:10093E00C3A861E524985002A824C3E89563400239
:10094E00A86388258826E570B4070375BB1E22743C
:10095E003279A787F0A4C5F0A2F733F8C3E8956102
:10096E004002A861882288248825882688642275FA
:10097E0040007541F022C2AF75C820A8CCA9CDAAFF
:10098E003A30CF010A75C824D2AFAB3BAC3C883BA2
:10099E00893CC3E89BF8E99C206908F9306702415D
:1009AE009021EDAD3D8A3DF9EA9DFA600478FF791C
:1009BE00FFAE3EAF3F8B3E8C3FA83BA93CC3E89EAB
:1009CE00F8E99FF9C3E54113FBE54013FAE82AF570
:1009DE0040E93BF54150067540FF7541FF4137AA8E
:1009EE0040AB41AC40AD417E047F02C3EB9404406A
:1009FE00021E1FC3EB940840021E1FC3ED13FDEC35
:100A0E0013FCDEF7C3EA9CFAEB9DFBEF6009C3E92A
:100A1E0013F9E813F8DFF7EA28FAEB39FB8A408B73
:100A2E004150067BFF8B408B41C3EB94025002D2A8
:100A3E00673069047F0341627892E6FFC3E537941D
:100A4E008240110FC3E53794A040010FC3EF940607
:100A5E0040027F057E02E541C4540FF9E541C454BE
:100A6E00F0F8E540C4540F28F8C3E89EFAE9940064
:100A7E00FB4009C3EA9402EB940050047A02E4FBB3
:100A8E0041DCAA40AB41EBC4FEEAC4540F4EFCC39A
:100A9E00EA9CFAEB9400FBC3E813C313F8EA28FAB6
:100AAE00EB3400FB8A408B41C3EB94024002C267D9
:100ABE007802EBC4FE7B00EAC4540F4EFAC3EA98E8
:100ACE00FA4005C3940250027A027892E6FF306033
:100ADE000241DC855192855293D26043E680C3E495
:100AEE009AF8E49BF93067026168E8FAE9FBD3E90A
:100AFE0013FDE813FC88518952C3EF94036038EF5D
:100B0E0020E00DE82CF8E93DF9ECFAEDFB020B3193
:100B1E00E828F8E939F9C3E82402F8E93400F97A4B
:100B2E00FE7BFFC3EF9403400E8A538B54884D898E
:100B3E004E8C4F8D50619C885389548A4D8B4E8CB0
:100B4E004F8D503069127553F07554FF754FF07517
:100B5E0050FF7551F07552FF619CE8FAD3E813FC13
:100B6E008851C3EF94036020EF20E007E82CF8ECE7
:100B7E00FA6188E8282402F87AFEC3EF940340084D
:100B8E008A53884D8C4F619C88538A4D8C4FE568F3
:100B9E00C3335002646BF56830600261A67534028F
:100BAE00D26043E680E52D54066034A840A941C3C7
:100BBE00E913F9E813F8C3E913F9E813F8306904F7
:100BCE00E92440F9C2AF53E67F759100C3E498F56E
:100BDE0094E499F595759104D26043E680D2AF22E4
:100BEE00D265754300752000306C03752040020CF1
:100BFE000DD265754300752040306C03752000786A
:100C0E00017901206720E52D54066002C265791432
:100C1E00E541C313700104F8C394144002781430F4
:100C2E006904781B791B206010E543600C30690362
:100C3E00D53404D26D81B871AE0543E59E7005E5DD
:100C4E009B020C54E59A5440B5200281A2306909EA
:100C5E0008C3E899400118813420650A08C3E89951
:0D0C6E004002810D8134C265C2AF53E67FA4
:100C7B007591003067127594007595FE759104D2CD
:100C8B006043E680D2AF810DAE40AF41C3E49EF529
:100C9B0094E49FF5958187C3E53394015002810D50
:100CAB00306502810DD80281B68134C26DC2AF535B
:100CBB00E67F759100855394855495759104854D08
:100CCB0092854E93D26043E680D2AFE52D540660F9
:100CDB0008206A020533020CF4306D0D206C0A20DB
:100CEB006507158115810215A62278003064053041
:100CFB0065027801E53775F007A4F9E5F028F5F002
:100D0B00E9A2F013A2F113A2F213F537C3947850B2
:100D1B0003753778C3E53795384008D266C293C25E
:100D2B0095C297306002A12E854F92855093D26069
:100D3B0043E68022207D19C2AF754202C294D29243
:100D4B00306202D297D2AF759F33759E00020F406F
:100D5B00C2AF754202C294D296306202D293D2AF26
:100D6B00759F33759E00020F40307243207D20C269
:100D7B00AF75420390013A757B10C297C2963062F1
:100D8B0004D295A192D294D2AF759E23020F40C28A
:100D9B00AF75420390013A757B10C293C2923062D9
:100DAB0004D295A1B2D294D2AF759E22020F4020ED
:100DBB007D17C2AF754203900115C297306202D204
:100DCB0095D2AF759E23020F40C2AF7542039001BF
:100DDB0015C293306202D295D2AF759E22020F409C
:100DEB00207D16C2AF754204C292D296306202D2F7
:100DFB0095D2AF759E22020F40C2AF754204C296C8
:100E0B00D292306202D295D2AF759E23020F403040
:100E1B007249207D23C2AF754205900129757B0471
:100E2B00C295C294306204D293C138D292D2AF75BC
:100E3B009F33759E00020F40C2AF75420590014B68
:100E4B00757B40C295C294306204D297C15BD29637
:100E5B00D2AF759F33759E00020F40207D1AC2AF33
:100E6B0075420590010BC295306202D293D2AF75D9
:100E7B009F33759E00020F40C2AF75420590011F54
:100E8B00C2953062E8D297D2AF759F33759E000240
:100E9B000F40207D16C2AF754206C296D2943062C7
:100EAB0002D293D2AF759E23020F40C2AF7542069A
:100EBB00C292D294306202D297D2AF759E22020FA9
:100ECB0040307243207D20C2AF75420190014B75BB
:100EDB007B40C293C292306204D297C1EAD296D2BF
:100EEB00AF759E22020F40C2AF754201900129756A
:100EFB007B04C297C296306204D293E10AD292D29B
:100F0B00AF759E23020F40207D17C2AF7542019033
:100F1B00011FC293306202D297D2AF759E22020F8D
:100F2B0040C2AF75420190010BC297306202D2935F
:100F3B00D2AF759E23C26622900109757B00C293C6
:100F4B00C295C297C292C294C296C2622278807630
:100F5B00090876090876040876FF0876030876FFF9
:100F6B00087607087603087601087601788C7601F7
:100F7B000876FF0876FF0876FF0876FF0876FF08ED
:100F8B0076030876FF0876FF0876FF087625087645
:100F9B00D00876280876500876040876FF08760283
:100FAB0008760008767A0876FF087601087601083D
:100FBB007600087603087600227887E6FFC272BFB8
:100FCB000302D2727888E6C394036008C27DE630D0
:100FDB00E102D27DC27E7889E630E102D27EC3EF98
:100FEB0094026008758E01D273020FFC758E00C2DD
:100FFB0073227880E6149000809378A5F67881E6CA
:10100B00149000809378A6F67886E61490008D9362
:10101B0078A7F67886E6F539C39402500375390242
:10102B00789CE67538FFB402037538A0B4030375DA
:10103B00388278A3E61490009A93F566120F432238
:10104B00227896E6FA7897E6FB7888E6B40305C330
:10105B00EB940EFB307F047A007BFFC3EB9AFCC34F
:0F106B00948250027C827572000572EC8572F0DF
:10107A00A4C3E5F0947D40F222D27F114C1205AE52
:10108A007A007B007C101205A4E55C2AFA74003B06
:10109A00FBDCF37C04C3EB13FBEA13FADCF7FEC2B6
:1010AA007F114C22E5EF20E6037520000520903DD4
:1010BA00FFE520146006901FFF146000930460038C
:1010CA0075EF1253D9BF7581C043FF8012059F7512
:1010DA00EF0243B203E5B3240220E70DF521E5B19F
:1010EA0020E0068521B343B101120F4375800875CC
:1010FA00A40075F1FF75D4F775900275A5FC75F219
:10110A00FC75D50075A0FD75A60275F30275D600AB
:10111A0075B0FF75A70175F4FF75E241120F43E43C
:10112A00F8F6D8FD756801120F581215F7789886E7
:10113A0073753001C2AF1205B81205C81205AE1296
:10114A0005CF1205AE1205D61205AEC2AF78FA79EE
:10115A00FA308307D9FBD8F7021C00120FC4120F0A
:10116A00FD114B114C78988673120F4375881075D0
:10117A00890275C82475910475D84075A82275B876
:10118A000275E690759B80759D00759A80759C0026
:10119A0075D10E75BC5875BB0175BA1F75E88012FA
:1011AA00059FD2AF1208BD75360053DACF207E03F1
:1011BA0043DA20307E0343DA1043DA01C2D8C2711F
:1011CA001205B8D2617B037A0CE55B70077A0CDBF7
:1011DA00030211551205AE207003021155C270E5C3
:1011EA005CC3940240E1E52F541F855E5DF55EB550
:1011FA005DD5DAD5C26153DACF207E0343DA2030D7
:10120A007E0343DA10C2D8C27178A2E67008D2749B
:10121A00E52F54E0F52FC2757529001205B3307415
:10122A0009C3E529940A4002D2751205A47802304E
:10123A0074027800C3E55C9840F0C2AF1205C81288
:10124A0005C81205C8D2AF1205B8754C007888E6F1
:10125A00B4030261331205A4788CE6C394015003E7
:10126A00021333E530C3940150030213332074355B
:10127A00C3E55C94FF5003021333C2AF1205DDD2FB
:10128A00AF1205B3C3E55C940150EFC2AF1205C8B3
:10129A001205A91205C8D2AF1205B3C3E55C94FFC3
:1012AA0040E902179F7F02D27F114C1205B3C2AFE9
:1012BA00C27F114CAE5CC3E55C947FD2AF4074121E
:1012CA00059FC2AF1205DDD2AFDFDC1183C3EE7812
:1012DA0097F61205B81216391217227F0AD27F1111
:1012EA004C1205B3C2AFC27F114CAE5CC3E55C942D
:1012FA007FD2AF50E612059FC2AF1205C81205A9E8
:10130A001205C8D2AFDFD61183EE24037896F612FF
:10131A0005B81216391217511205B3114CC3E55C00
:10132A0094FF5002417702179FC3E55C954C400336
:10133A00855C4C1205B378017988E7B40302780515
:10134A00C3E55C9840024157C2AF1205DD1205DDC4
:10135A001205DDD2AF1205B8753000E4F531F53269
:10136A000531E531F4703F0532789AE67819146050
:10137A0012783214600D787D14600878FA146003CC
:10138A00753200C3E53298401D120F4312059F15AE
:10139A003275310078998673C2AF1205DDD2AF7803
:1013AA009886731205B31205A9E52A7005307402EE
:1013BA00215578012074027806C3E55C9840A1782B
:1013CA0088E6C3940360031205B3E52A7003021189
:1013DA0055C2AF120F43E4F522F523F524F525F59E
:1013EA0026F567D2AF7885E6C333F565E4F544F5AB
:1013FA0045F546F547F548F570F52CF52DF53775A1
:10140A00700875BB1E12059F1208C1E5E820ECFBA7
:10141A00A8BDA9BEE97001F888711208C5757008DF
:10142A0075BB1E120FC4C2AF7561FF12095D85221A
:10143A0061852262852263D2AF7522017524017506
:10144A002501752601856069756A017888E6B40305
:10145A0007C27D307602D27DD268D2697533001216
:0E146A000E9D120ECC12097D12098412097D0E
:1014780012098412097D120BFF1206B8120CF5121C
:101488000D3F120984120BEE306E03120714206709
:10149800031208603067031208A7120CF5120D74C6
:1014A800120984120BFF306E03120749120CF51251
:1014B8000DEB120984120BEE306E031207A7120C03
:1014C800F5120E1A120984120BFF306E031208046B
:1014D800120CF5120E9D1209841208C1120BEE129D
:1014E8000CF5120ECC1208C51209843069328564D5
:1014F80061856462856069756A0179187A0CC3E54B
:101508003399400FC269D26A8A35856461856463FC
:10151800021528C3E55C9401400302147E0215AE4F
:10152800306A1D206C1AE535147006C26AD26B81C8
:101538007EF535C3E55C9401400302147E0215AEC6
:1015480075360078FA79A4E760027803C3E55F98F6
:101558005054307404E52A604D7888E6B4031720A7
:101568007D05207607A17E307602A17E206C07D209
:101578006C85646181BD78F0306C05856461782084
:10158800C3E541985002817E306C1BC26CC27D302D
:101598007602D27DD26A753512856461817E053600
:1015A800E55C6002A1B1753600C2AF120F437887BF
:1015B800E6FE7602120FC47887EEF6E4F522F523EC
:1015C800F524F525F526F565752C00752D00D2AFA7
:1015D8001205B3120F4378A4E66006D293D295D2CF
:1015E80097307409C3E5369404400221556165902B
:1015F8001A0D782012167BE520B4550CA312167B21
:10160800E520B4AA03021619120F58121639021649
:1016180038901A0378807B0A12167BA308DBF990AE
:101628001A0F788C7B1912167BA308DBF9901A28FD
:1016380022C2AF1216BA121694901A00740E12161D
:1016480080A37406121680A37415121680901A03CC
:1016580078807B0A12167FA308DBF9901A0F788C22
:101668007B1912167FA308DBF91216CD1216AB9060
:101678001A2822E493F622E6438F01538FFD75EF73
:101688000275B7A575B7F1F0538FFE22438F024359
:101698008F0175EF0275B7A575B7F1901A0DF05364
:1016A8008FFC22901A0D7455D180901A0E74AAD10D
:1016B80080227A3079D07820901A40D17BE520F7C3
:1016C80009A3DAF7227A3079D0901A40E7D1800955
:1016D800A3DAF922AB74A875BB01027980BB0202B8
:1016E8007981BB03027982BB04027984BB05027944
:1016F80086BB06027992BB07027987BB080279A3E9
:10170800BB0902799CBB0A027988BB0B027989E87C
:10171800F7227C051205B8DCFB22C2AF1205C812FD
:1017280005CF1205D61205DD1205A91205C8120546
:10173800CF1205D61205DD1205A91205C81205CF6C
:101748001205D61205DDD2AF22C2AF1205DD120591
:10175800D61205CF1205C81205A91205DD1205D645
:101768001205CF1205C81205A91205DD1205D612F9
:1017780005CF1205C8D2AF22AE74AF75C2AF12053D
:10178800C81205C81205C81205A9DEF21205DD1235
:1017980005A9DFF8D2AF22F122F11AF11A75740106
:1017A800757501757600F1807C05AD5C1205B8C3CE
:1017B800ED955C70F5C3E55C9401400AC3E55C9463
:1017C800FF40320217DBD1DCD139F122C2AF75EF0D
:1017D80012F11ADCD50576C3E5769403500280C66B
:1017E800F11A0575E5741490009F93F808C3E57520
:1017F80098500280AEF11A12171A0574C3E5749452
:101808000C5002809B120F58121639C2AF75EF1296
:0318180012171A8A
:0319FD000210AE27
:101A00000E0615090904FF03FF0703010155AA018A
:101A1000FFFFFFFFFF03FFFFFF25D0285004FF0259
:091A2000007AFF0101000300FF40
:101A400023506C6174696E756D31353041232020EF
:101A500023424C48454C4923463331302320202033
:101A60002020202020202020202020202020202076
:101C0000C2AFC2D353D9BF7581C043B20343FF8073
:101C1000752438752503B1C975EF0275E24043F1AB
:101C20000853A4F775D4FFD2837DFA780379E67C54
:101C300010752200752300901DD67B0675249875BB
:101C400025013083028142208308D8FBD9F9DCF7D3
:101C500081B4308308D8FBD9F9DCF781B4B189E4C9
:101C600093A3C39A6004DDC381B4DBDBB17B600264
:101C7000812B7B08E493FAA3B15CDBF87A30B15C8A
:101C8000752200752300B17BEAFCEBFDC3ED94FEE9
:101C9000400EB17B8A278B28ED30E0048A828B834B
:101CA000B17B7AC270D8C3ED94FE601350CEBD00F4
:101CB00025EC60097520007521FF0200008100A855
:101CC00027A9280809D804D90281D3B17FEA89AAB3
:101CD000F281C50D81A0C3ED94035049EDA2E092BD
:101CE000007AC5C3E5829400E583941C50902000DF
:101CF00010438F02438F0175B7A575B7F1F030001F
:101D00001FA827A9280809438F01538FFDD804D99C
:101D100002A12089AAE275B7A575B7F1F0A3A10DBC
:101D2000538FFC817C7AC1BD030CE493A3FAB140CC
:101D3000DCF8B138817C817EAA22AB23B15CEBFA5E
:101D4000EA6222752608C3E52313F523E52213F57D
:101D50002250066323A0632201D526EAB1C9B1C986
:101D600075260AEAF4200102D283300102C283B14F
:101D7000C9C3134002C201D526EB22B17FEAFB2082
:101D80008302A17F308302A184752608AE24AF258B
:101D9000C3EF13FFEE13FEB1CDB1C9C3EA13308315
:101DA000024480FA30E703632201C3E52313F523DD
:101DB000E52213F52250066323A0632201D526D91C
:101DC000E52265236523F52222AE24AF250E0FDE22
:101DD000FEDFFCD20122424C48656C693437316326
:041DE000F3100601F5
:00000001FF
